:020000001E28B8
:080008000B110900F4000030A7
:100010008A000F30740703188A0A740882070730B1
:100020008A004D2F07308A00662F07308A007F2F05
:1000300007308A00982F07308A00B12F20308312B2
:100040000313B6000430B7000230B800CC018312AD
:100050000313CD010930CE000130CF00D000D10014
:100060000230D2000830D3000130D4002030D50057
:1000700046230130C800F026FE01D5260230831247
:100080000313C800F0260330FE00D526FA30831291
:100090000313B4000627FA30B4000627A526023061
:1000A00083120313C800F0260630FE00D5268123F4
:1000B0008123831203130608F000F00CF00CF00CFF
:1000C000700C0F39F0007008063C031D7128831274
:1000D0000313A001A101A201A3018F30A400662394
:1000E000C6297008073C031DEE2801308312031354
:1000F0005102031DAB2805304D02013003180301E6
:10010000F1004D08073C0130031803017104003C65
:100110000319A4284D08093C013003190301F1001B
:100120004D080B3C0130031903017105003C031914
:10013000A4284D08A000A101A201A3010730A4003A
:10014000662383120313CA00CD0A0D304D02031D2E
:10015000C629CD01C6290230831203135102031DA3
:10016000D42801305402031DB8280230D400ED28F1
:1001700002305402031DBF280330D400D3280330BB
:100180005402031DC6280430D400D328043054027E
:10019000031DCD280530D400D32805305402031D9B
:1001A000D3280130D400ED28033083120313510209
:1001B000031DED28A001A101A201A3015308A40081
:1001C000662383120313CA0008305302031DEB2871
:1001D0008830D300ED280830D300C62970080B3CC6
:1001E000031D31290130831203135102031D0B2912
:1001F0000F304F02031DFE280130CF004F08BC0016
:100200004224013083120313A400662383120313D4
:10021000CA00CF0AC62902305102031D1A29C001A3
:100220005408C1000C250130A40066238312031377
:10023000CA00302903305102031D3029A001A10159
:10024000A201A3015208A400662383120313CA006B
:10025000CA08031D2E298230D20030290230D20074
:10026000C62970080D3C031D7C290130831203133D
:100270005102031D4629A001A101A201A301813061
:10028000A400662383120313CA00C6290230510258
:10029000031D56290130C0005408C1000C2501304F
:1002A000A400662383120313CA007B290330510282
:1002B000031D7B294E08A000A101A201A301093062
:1002C000A400662383120313CA0009304E02031DE3
:1002D0006E294930CE002D30D5007B2949304E02A1
:1002E000031D77298930CE002B30D5007B290930BA
:1002F000CE002030D500C62970080E3C031DC6294B
:100300000430831203135002031D88290130D000EA
:100310003230B40006275008F1007108013C031D7B
:100320009E29023083120313C800F0260630FE0017
:10033000D526013083120313D100C1297108023C74
:10034000031DAF29023083120313C800F0260930C1
:10035000FE00D526023083120313D100C129710893
:10036000033C031DC129023083120313C800F02689
:100370000C30FE00D526033083120313D100C129AF
:10038000C12983120313D00AC629C6298312031375
:10039000C9012227553083120313C9002227831273
:1003A0000313C901222783120313C9012227BB307B
:1003B00083120313C90022273127FC003127FD00D7
:1003C0007C080139031DED29013083120313BD00A0
:1003D000BE014130BF00FE24F52901308312031312
:1003E000BD00BE014230BF00FE247C084039003C05
:1003F0000319022A013083120313BD00BE014D30E0
:10040000BF00FE248123F0013030F1002508F20006
:10041000F20CF20CF20C720C0F3971070318F00A8F
:10042000AA00303C031D162A2030AA00F00130300B
:10043000F1002508F200720EF039F039F200F20CEA
:10044000F20CF20C720C0F3971070318F00AAB00B2
:100450002A08203C0130031D0301F0002B08303C2A
:100460000130031D03017005003C0319392A2030B7
:10047000AB00F0013030F1002608F200F20CF20C73
:10048000F20C720C0F3971070318F00AAC002E3011
:10049000AD00F0013030F1002608F200720EF039A4
:1004A000F039F200F20CF20CF20C720C0F397107F9
:1004B0000318F00AAE00F0013030F1002708F20016
:1004C000F20CF20CF20C720C0F3971070318F00ADF
:1004D000AF00F0013030F1002708F200720EF03961
:1004E000F039F200F20CF20CF20C720C0F397107B9
:1004F0000318F00AB0002E30B100F0013030F100E6
:100500002808F200F20CF20CF20C720C0F39710791
:100510000318F00AB200F0013030F1002808F200B0
:10052000720EF039F039F200F20CF20CF20C720C8F
:100530000F3971070318F00AB3004C08093C031C7B
:10054000B62A0130BD00F00102304C070318F00A52
:10055000BE004C082A3E8400831300088312031354
:10056000BF00FE2483120313CC0A9D2ACC01013064
:10057000BD000C30BE005508BF00FE2401308312C0
:100580000313B9000D30BA002908BB00AB23A0014A
:10059000A101A201A301F730A40066238312031373
:1005A000CA008039031DDB2A0230BD00BE01503075
:1005B000BF00FE24F82A023083120313BD00BE01DF
:1005C0007330BF00FE2483120313A001A101A20116
:1005D000A301E730A400662383120313CA00803905
:1005E000031DF82A0230BD00BE015330BF00FE24B7
:1005F000831203134A08F000700EF039F039F0004E
:10060000F00CF00CF00C700C0F39CB0001304B02E9
:10061000031C2F2B01304B020130031C0301F0009F
:100620004B08093C0130031C03017005003C031911
:10063000252B0230BD000130BE00F00130304B07E9
:100640000318F00ABF00FE24382B02308312031374
:10065000BD000130BE002B30BF00FE24382B02301D
:1006600083120313BD000130BE002030BF00FE2402
:10067000023083120313BD000630BE00F00130309B
:1006800054070318F00ABF00FE24592804308312CF
:10069000031386008316F03083168500F23086003F
:1006A0004030810083128B016026A526073083121B
:1006B00003139F0083161930831699002430980085
:1006C00083129030831298008C0108008312031368
:1006D0002008C9002227831203132108C9002227FA
:1006E000831203132208C90022278312031323084D
:1006F000C9002227831203132408C90022273127A7
:10070000080083120313C901222783120313C901AE
:10071000222783120313C901222783120313C9015D
:100720002227033083120313C900222731278312A3
:100730000313A500312783120313A6003127831268
:100740000313A700312783120313A8003127831254
:100750000313A900080083120313D9013B08F0001A
:100760007008003C031DBD2B4C3083120313D600D0
:100770005330D7004230D800262C7008013C031DAE
:10078000CA2B553083120313D6005330D7004230A2
:10079000D800262C7008023C031DD72B2030831272
:1007A0000313D6004330D7005730D800262C7008EA
:1007B000033C031DE42B433083120313D600573050
:1007C000D7005230D800262C7008043C031DF12BB2
:1007D000203083120313D6004130D7004D30D800AB
:1007E000262C7008063C031DFE2B57308312031382
:1007F000D6004630D7004D30D800262C7008083C73
:10080000031D0B2C203083120313D6004630D70073
:100810004D30D800262C70080A3C031D182C44309B
:1008200083120313D6004930D7004730D800262C56
:1008300070080C3C031D262C503083120313D60085
:100840004B30D7005430D800262C262C83120313AB
:100850005908023C031C412C3908BD00F0013A083C
:1008600059070318F00ABE005908563E8400831346
:10087000000883120313BF00FE2483120313D90A56
:10088000262C0800831203133C08F1007108013C78
:10089000031D522C433083120313A000A101A201B7
:1008A000A301FD2C7108023C031D5F2C1430831240
:1008B0000313A0005030A100A201A301FD2C710878
:1008C000033C031D6C2C113083120313A0008030F5
:1008D000A100A201A301FD2C7108043C031D792C89
:1008E000083083120313A0008030A100A201A301ED
:1008F000FD2C7108053C031D872C05308312031362
:10090000A0000130A1005030A200A301FD2C71080D
:10091000063C031D942C023083120313A000843084
:10092000A100A201A301FD2C7108073C031DA12C0D
:10093000023083120313A0004230A100A201A301E0
:10094000FD2C7108083C031DAE2C023083120313EA
:10095000A0001430A100A201A301FD2C7108093CE4
:10096000031DBB2C013083120313A0008230A100B1
:10097000A201A301FD2C71080A3C031DC82C013003
:1009800083120313A0004230A100A201A301FD2C99
:1009900071080B3C031DD52C013083120313A000FA
:1009A000A1015030A200A301FD2C71080C3C031DD5
:1009B000E22C83120313A0017030A1005030A2007A
:1009C000A301FD2C71080D3C031DEF2C83120313B2
:1009D000A0013630A1004030A200A301FD2C710817
:1009E0000E3C031DFD2C83120313A0011830A1003F
:1009F0004030A200A301FD2CFD2C0800831203133C
:100A00003D08C6003E08C700B12683120313061432
:100A10003F08C5008E26080083120313DC019930BD
:100A2000DD002508D6002608D7002708D8002808AA
:100A3000D9004008003C0319222D5D08DA005C084B
:100A4000DB00262D5C08DA005D08DB000130410286
:100A5000031D6D2D59085A02031D622D5B08D90034
:100A600058085A02031D572D5B08D80057085A0230
:100A7000031D4C2D5B08D70056085A02031D432D59
:100A80005B08D600B12D5608C2004008C3000130F3
:100A9000C400BA25D600B12D831203135708C20033
:100AA0004008C3000130C400BA25D700B12D83121D
:100AB00003135808C2004008C3000130C400BA251F
:100AC000D800B12D831203135908C2004008C30097
:100AD0000130C400BA25D900B12D023083120313AE
:100AE0004102031D7C2D5708C2004008C30010308E
:100AF000C400BA25D700B12D03304102031D892D52
:100B00005708C2004008C3000130C400BA25D7000E
:100B1000B12D04304102031DA52D5808C200400824
:100B2000C3000230C400BA25D800C2004008C30088
:100B30001030C400BA25D8005908C2004008C300CC
:100B40005030C400BA25D900B12D05304102031D33
:100B5000B12D5808C2004008C3000530C400BA25B2
:100B6000D8005608A0005708A1005808A20059084C
:100B7000A3000800831203134308003C0319152E39
:100B800042080A3C013003190301F10042081A3CF3
:100B90000130031903017105F10042082A3C0130BC
:100BA000031903017105F10042083A3C01300319B1
:100BB00003017105F10042084A3C013003190301A9
:100BC0007105F10042085A3C013003190301710517
:100BD000F10042086A3C0130031903017105F1007C
:100BE00042087A3C0130031903017105F100420803
:100BF0008A3C0130031903017105F10042089A3C57
:100C00000130031903017105003C03190E2EF10197
:100C1000420844070318F10AC2005E2EF10142089F
:100C2000073E0318F10AC2005E2E83120313420826
:100C3000103C013003190301F1004208203C01304F
:100C4000031903017105F1004208303C013003191A
:100C500003017105F1004208403C01300319030112
:100C60007105F1004208503C013003190301710580
:100C7000F1004208603C0130031903017105F100E5
:100C80004208703C0130031903017105F10042086C
:100C9000803C0130031903017105F1004208903CCA
:100CA0000130031903017105003C03195B2E440850
:100CB0004202C2005E2E07304202C2004208080013
:100CC0008312031306100530B40006270330850095
:100CD000A0260530B400062702308500A026053086
:100CE000B40006272830C5008E2601308312031376
:100CF000B40006270830C5008E2601308312031386
:100D0000B40006270C30C5008E2601308312031371
:100D1000B40006270630C5008E2608008312031390
:100D20004508F200F20CF20CF20C720C0F3985003F
:100D3000A02645088500A0262830FF0017270800B8
:100D400083120313861586110800831203130610FD
:100D50000130C5008E26023083120313B40006272B
:100D6000080083120313061001304602031DC02E33
:100D7000F001803047070318F00AC5008E26CF2EF9
:100D8000F00140308312031347070318F00AF10003
:100D900070080038F00071088038C5008E260230D7
:100DA00083120313B4000627080083120313D6012D
:100DB0000614831203135608F3007E080620FF3939
:100DC000003C0319EF2E831203135608D60AF300D2
:100DD0007E08062083120313C5008E26D92E080034
:100DE00083120313061001304802031DFB2E8030CE
:100DF000C5008E26002FC03083120313C5008E2637
:100E0000023083120313B400062708008E308312C9
:100E10000313B50000000000000000000000000007
:100E2000B50B0C2F0000B40B062F00000800FF0CC0
:100E3000FF0C3F30FF050330FF020000FF0B1D2FAA
:100E400000000800831203134908990083168312D7
:100E50000313010803192F2F83161808272F831255
:100E60000800831203130C083605FF39003C0319F0
:100E7000312F18083705FF39F10018083805FF39F8
:100E80007104003C0319492F1812000018161A08A3
:100E9000DE001A080800312F080007308A0055309C
:100EA000730703188A0A73088207463454342D34B2
:100EB0003834313437342034523465346D346F343F
:100EC000743465344D3461346E34003407308A0034
:100ED0006E30730703188A0A73088207493457343F
:100EE00032344C34463444342034723431342E3469
:100EF0003034203432343034303434340034073039
:100F00008A008730730703188A0A7308820720341F
:100F100020342034203420342034203420345634FB
:100F2000663420344234643420344D346434003424
:100F300007308A00A030730703188A0A73088207F3
:100F40002034203420342034203420342034203401
:100F5000553470342034443477342034533474346A
:100F6000003407308A00B930730703188A0A7308FF
:100F7000820720342034203420342034203420349C
:100F8000203452347034203453347034203450348C
:040F900054340034A1
:02400E00503F21
:00000001FF
